:020000040800F2
:1000000000040020E1010008610D0008610D0008F6
:10001000610D0008610D0008610D0008610D000808
:10002000610D0008610D0008610D00087D2E0008BB
:10003000610D0008610D0008610D0008610D0008E8
:10004000610D0008610D0008610D0008610D0008D8
:10005000610D0008610D0008610D0008610D0008C8
:10006000610D0008610D0008610D0008610D0008B8
:10007000610D0008610D0008610D0008610D0008A8
:10008000610D0008610D0008610D0008610D000898
:10009000610D0008610D0008610D0008610D000888
:1000A000610D0008610D0008610D0008610D000878
:1000B000610D0008610D0008610D0008610D000868
:1000C000610D0008610D0008610D0008610D000858
:1000D000610D0008610D000815260008610D00087B
:1000E000610D0008610D0008610D0008610D000838
:1000F000610D0008610D0008610D0008610D000828
:10010000610D0008610D000899250008610D0008C7
:10011000610D0008610D0008610D0008610D000807
:10012000610D0008610D0008610D0008610D0008F7
:10013000610D0008610D0008610D0008610D0008E7
:10014000610D0008610D0008610D000845230008DD
:10015000610D0008610D0008610D0008610D0008C7
:10016000610D0008610D0008610D0008610D0008B7
:10017000610D0008610D0008610D0008610D0008A7
:10018000610D0008610D0008610D0008610D000897
:10019000610D0008610D0008610D0008610D000887
:1001A000610D0008610D0008610D0008610D000877
:1001B000610D0008610D0008610D0008610D000867
:1001C000610D0008610D0008610D0008610D000857
:1001D000610D0008610D0008610D0008610D000847
:1001E00072B6374880F3098836484EF60851CEF289
:1001F0000001086040F20000CCF200004EF63471BD
:10020000CEF200010860BFF34F8FBFF36F8F40F253
:100210000000C0F2F0004EF68851CEF200010860F6
:10022000BFF34F8FBFF36F8F4FF00000E1EE100A66
:100230004EF63C71CEF200010860062080F314886F
:10024000BFF36F8F00F06EFD02F0DAFA1E481F490F
:100250001F4A91423CBF41F8040BFAE71D49184A76
:1002600091423CBF41F8040BFAE71B491B4A1C4B67
:100270009A423EBF51F8040B42F8040BF8E7002005
:100280001849194A91423CBF41F8040BFAE700F0C3
:100290004DFD02F0B7FA154C154DAC4203DA54F897
:1002A000041B8847F9E700F041F8124C124DAC42AC
:1002B00003DA54F8041B8847F9E700F035BD000065
:1002C000000800200000000855555555000000208A
:1002D0000004002000040020D83B00080008002093
:1002E0002808002028080020A8220020E00100089B
:1002F000E0010008E0010008E00100082DE9F04FEE
:100300002DED108AC1F80CD0C3689D46BDEC108A53
:10031000BDE8F08F002383F311882846A047002012
:1003200000F038FF00F0DCFE00DFFEE738B5184BC8
:1003300014221A706FF03F0200245A720F225C7070
:100340009C70DC701C715C719C71DC711C729A7207
:10035000DC7202F0B5FC0F4B984208D00133984292
:1003600041F2883412BF00250024012500E0254613
:10037000002002F0ABFC0DB100F052F800F076FC6A
:1003800000F040FB204600F091F800F049F8F9E752
:1003900028080020010007B008B500F0BDFAA0F160
:1003A00020035842584108BD07B5054B01A81B88DA
:1003B000ADF80430022100F00FFB03B05DF804FB40
:1003C0007038000808B51248C3680BB100F094FDFE
:1003D000104A0F4800234FF47A7100F051FD0E4B84
:1003E0001A6812B11A68013A1A605A680A4912B1B9
:1003F0004A68013A4A60094A12783AB95B682BB9EF
:10040000022000F0E5FB044B32225A6008BD00BF19
:1004100034080020C50300084C0D0020480D0020C2
:1004200038B51B4C2368013330D01A4D1A4B2A685B
:100430009A422BD9194B9B6803F1006303F5804363
:100440009A4223D2002000F0F7FA154B02201870D0
:1004500000F0B0FB134B1A6C00221A64596C5A64FA
:10046000596941F0800159615A61196941F000519F
:1004700019611A6172B60C4B1C6023682A6820212E
:1004800081F311889D4683F30888104738BD00BF6B
:100490000040000804400008FF3F00082808002032
:1004A000480D00200038024008ED00E02DE9F04F33
:1004B000BE4B8046BE489C680022C26091B020229C
:1004C00082F31188C26801930AB100F015FDB848A3
:1004D000B84A4FF47A71002300F0D2FC002383F372
:1004E0001188DFF8ECA2B8F1000F01D0CAF8008043
:1004F000B14ECAF8043000253370A9464FF0FF37DB
:10050000012000F057FBB8F1000F04D0DAF80030FA
:10051000002B00F0F781002000F0FEF90590059B0C
:10052000002BF0DB012000F039FB059B213B122B57
:10053000E6D801A252F823F08505000897050008C7
:100540000306000801050008010500080105000870
:10055000770600080105000827070008D5070008EE
:10056000030800082D0800080105000843080008DA
:10057000010500086D080008D10800080105000801
:100580009D0800080220FFF707FF002800F0A78160
:100590004FF001099CE14FF47A7000F0BDF9B0F121
:1005A000000BC0F29C810220FFF7F6FE002800F04D
:1005B00096810BF1FF30042800F29181DFE800F012
:1005C00003080A0C110010A8052340F8143D04E0AC
:1005D000764802E0794800E07948042100F0FCF90F
:1005E0000DE01C25284600F029FA10AB042143F841
:1005F000140D0435184600F0EFF92C2DF2D1012529
:1006000066E1B9F1000F00F06A81002D00F067810A
:100610000220FFF7C1FE10B90125A9465FE10120C4
:1006200000F00AFA0220307000F0C4FA0024E3B2AD
:100630001846029300F018FA01348346029B18B161
:10064000184600F021FAF2E701230220337000F08F
:10065000A5FA019B9B689B4508D2584600F0EEF92D
:10066000013040F045810BF1040BF2E700243470B7
:10067000CAF804402CE1B9F1000F00F03081002DE0
:1006800000F02D810220307000F094FA322000F04A
:1006900043F9B0F1000BBFDB1BF00303BCD10199A0
:1006A00089680BEB04028A42B6D8BBF5807FB3D8C9
:1006B0005B450EDA4FF47A70029300F02DF9059045
:1006C000059A002AA8DB029B3E4A059999540133FA
:1006D000EEE7C820FFF760FE00289DD024B9394B13
:1006E0004FF0FF321F681A602BF0030B0BEB040373
:1006F000A3469B4515D0334A0393121B584652F824
:100700000B10029200F0A0F9584600F097F9029AF7
:1007100052F80B20904240F0EB800BF1040B039B4E
:10072000E7E75C46D4E00220FFF736FE002800F041
:10073000D6804FF00008C346019B9B68984530D295
:10074000B8F1000F03D17A1C01D00B9703E04046AB
:1007500000F074F90B901C494B6893B91A460820B5
:1007600012F0010F4FEA520E16BF184A72468EEA77
:1007700002020138F4D141F823200133B3F5807F20
:10078000ECD100220BABD35C83EA0B03DBB201326A
:1007900051F82330042A83EA1B2BF3D108F1040813
:1007A000CAE710A840F828BD29E000BF28080020AB
:1007B00034080020C5030008480D00202C08002044
:1007C00030080020480C0020480800202083B8EDA5
:1007D0004C0D002010A8002340F8143D642100F0C7
:1007E000CDF800287BD10220FFF7D6FD002876D077
:1007F0000B9800F05BF910AB43F8240D1846042168
:1008000031E010A8002340F8143D642100F0B6F850
:10081000002864D10220FFF7BFFD00285FD00B98AD
:1008200000F054F910AB43F8200DE7E70220FFF782
:10083000B3FD002853D000F04FF910AB43F81C0D66
:10084000DCE70220FFF7A8FD002848D00BA9142000
:1008500000F048F9804610A8042140F8188D00F0F7
:10086000BBF80BA8414600F0B7F831E04FF47A70BE
:10087000FFF792FD98B37B1C05D1FFF795FD234848
:1008800000F08EFC3EE00020394600F0DDF800204C
:1008900000F0D4F8B842F0D0A34629E010A8002315
:1008A00040F8143D642100F069F88346B8B902208D
:1008B000FFF772FD98B1FFF777FD41F2883000F045
:1008C0006FFC0B9800F00CFAD84600F0C5F917E65B
:1008D00000F0C2F94FF00008FFF766FD10E60C4B80
:1008E0000BA81B88ADF82C30022100F075F807E644
:1008F000084B0BA81B88ADF82C30022100F06CF8D7
:100900005C46FDE511B0BDE8F08F00BFA086010098
:100910007238000874380008F7B500244FF47A756F
:100920008DF807404543124B93F900305A1CE6B24C
:1009300001D0A34210D10F4B53F8240003680DF1EE
:100940000701DF6901222B46B847012804D10A4B71
:100950009DF807001E7008E00CB90124E3E74FF48E
:10096000FA7000F01DFC4FF6FF7000B203B0F0BD4E
:100970000008002078380008680D0020F8B54FF412
:100980007A7506464D430024104B93F900305A1CEB
:10099000E7B201D0A3420FD10D4B53F824000368F6
:1009A0003146D3F81CC004222B46E047042803D16B
:1009B000084B1F700020F8BD0CB90124E4E74FF488
:1009C000FA7000F0EDFB4FF0FF30F8BD000800209A
:1009D00078380008680D002010B50A46064903461D
:1009E0000878064951F8200001688C691946A44628
:1009F000034BBDE810406047680D002078380008C0
:100A0000A086010070B502F085F8094B0026187029
:100A10001C46084D23782868984208D202F074F8E2
:100A20002B6806440133B6F5804F2B60F1D370BDBF
:100A3000700D00206C0D002002F02EB900F1006056
:100A400000F580400068704707B502AB00F1006018
:100A500043F8041D0422194600F5804002F09EF878
:100A600003B05DF804FB0000054B1A68054B1B78CA
:100A70001344984202D2104402F046B80020704756
:100A80006C0D0020700D002038B5074D0446286815
:100A9000204402F041F828B928682044BDE83840D5
:100AA00002F052B838BD00BF6C0D0020034610F0B4
:100AB000030008D1B3F5007F06D803F10053A3F576
:100AC000084318687047002070470000014BC05869
:100AD000704700BF107AFF1F014B1868704700BFB6
:100AE000002004E070B52A4B1C68C4F30B03240CEF
:100AF00083B140F21342934209D040F2194293422B
:100B000007D040F2214293420BD1032302E001239C
:100B100000E002231F4A0C2505FB03235D681A7AB7
:100B200001E01D4D3F2242F201039C422CD0B4F55E
:100B3000805F08D041F201039C420BD041F20303D5
:100B40009C4209D000E0412241F207039C4208BFC9
:100B5000312202E05A2200E05922461E0E44013D95
:100B60000C46B4420ED215F8010F631C18B11C4696
:100B700003F8010CF5E72C20B342207006D2A31C29
:100B8000627003E0234601E03322DDE7581A70BDAE
:100B9000002004E080380008B0380008022801D1A5
:100BA000082202E0012802D10422014B9A61704719
:100BB00000100240022802D14FF4002203E0012875
:100BC00003D14FF48022014B9A617047001002401C
:100BD000022804D1064A536983F0080305E001287E
:100BE00004D1034A536983F004035361704700BF83
:100BF0000010024010B50023934203D0CC5CC454D3
:100C00000133F9E710BD000030B5013810F8013F9D
:100C10000C4663B12578AB4201F1010107D10AB15D
:100C2000013AF3E75AB294F90030D01A30BD002AE5
:100C3000F8D1104630BD000002460346981A13F959
:100C4000011B0029FAD1704702440346934202D0A7
:100C500003F8011BFAE77047024B1A78024B1A702F
:100C6000704700BF680D00200008002038B5164D01
:100C7000164C284600F0C8FB2146284600F0F0FB41
:100C8000236813485A6DD2F8043843F00203C2F8BF
:100C9000043800F085FA20680E4900F0FFFC236854
:100CA0000D485A6D0D49D2F8043823F00203C2F8FA
:100CB0000438A8424FF4E1330B6003D0BDE838405C
:100CC00000F008BB38BD00BF60190020703B000871
:100CD00040420F00043B0008F0100020540D00209B
:100CE00038B50C4B1A780C4B53F822400B4B9C42F6
:100CF00005460DD00A4B002118461422FFF7A4FF29
:100D00000346056019462046BDE8384000F0E2BAC7
:100D100038BD00BF680D0020783800086019002039
:100D2000540D002070470000FEE70000084A094B00
:100D300009498B4204D252F8041F43F8041BF7E719
:100D4000064A934203D2002243F8042BF8E7704787
:100D5000FC3B0008A8220020A8220020A822002096
:100D60001EF0040F0CBFEFF30880EFF309808169D8
:100D7000004A10477D0D000870470000204B0268B4
:100D80001A60204B42681A601F4B82681A601F4B22
:100D9000C2681A601E4B02691A601E4B42691A60D3
:100DA0001D4B82691A601D4BC2691A601C4B1D499C
:100DB0001A681D4B1A601A68120A0A701A681B4BCF
:100DC0001A701B4B1A681B4B1A601B4B1A681B4B83
:100DD0001A601B4B1A681B4B1A601B4B1A681B4B83
:100DE0001A601B4B1A681B4B1A601B4B5A6A1B4B31
:100DF0001A601B4B1B68DB0701D500BEFEE7FEE750
:100E0000A80D0020AC0D0020B00D0020B40D002076
:100E1000840D0020740D0020800D00208C0D00201A
:100E200028ED00E0940D0020980D0020780D0020A2
:100E30002CED00E0A40D002030ED00E09C0D002022
:100E40003CED00E0900D002034ED00E0A00D00200E
:100E500038ED00E0880D002000ED00E07C0D002062
:100E6000F0ED00E0054B03F114025A619A614FF076
:100E7000FF32DA6100221A62704700BFB80D00200D
:100E8000F8B503611A4BC2605C6A1A4B1A46012915
:100E900098BF022152F8145F954206461F460AD1B8
:100EA000586198611C620560456081600819BDE861
:100EB000F84000F0CDBB186AAB68241A0C1905D2B3
:100EC0009C4205D2204400F0D3FB01E02D68E41AD7
:100ED000AB68A342FAD36B68736035601E606E60C6
:100EE000B460A9684FF0FF33091BA960FB61F8BD2E
:100EF000000C0040B80D002010B51A4C234653F8E2
:100F0000142F82420ED0416802680A600268516064
:100F10009A424FF00001C16022D0916883680B446F
:100F2000936010BD11686161002099424B60D060F0
:100F300003D1BDE8104000F095BB8B6892681A445D
:100F4000094B8A60586A236AC31A934208D2D31A9B
:100F5000012B98BF02231844BDE8104000F088BB65
:100F600010BD00BFB80D0020000C0040024B002255
:100F70001B605B609A607047B80D0020002303740B
:100F80008268054B1B6899689142FBD25A680360DE
:100F90004260106058607047B80D002008B52023EB
:100FA00083F31188037C032B03D0042B05D04BB9AA
:100FB0000EE0436900221A6004E090E80C001A6019
:100FC000026853604FF0FF334361FFF7D7FF002300
:100FD00083F3118808BD0000002303748268054B69
:100FE0001B6899689142FBD85A68036042601060A0
:100FF00058607047B80D0020054B196908741868CF
:1010000002681A605360186101230374FFF776B910
:10101000B80D002030B54B1C87B005460A4C0DD0EA
:1010200023690A4A01A8FFF72BFF2846FFF7E4FFD0
:10103000049B2BB101A8FFF75FFF01E0FFF7DCFF86
:101040002369586907B030BDB80D00209D0F000816
:1010500038B50C4D41612B6981689A68914204460C
:1010600003D8BDE83840FFF789BF1846FFF786FF71
:1010700001232C61014623742046BDE83840FFF768
:101080003DB900BFB80D0020044B1A681B69906879
:101090009B68984294BF002001207047B80D002043
:1010A00010B5084C236820691A6822605460012238
:1010B00023611A74FFF790FF01462069BDE81040D4
:1010C000FFF71CB9B80D0020044B1A681B69926821
:1010D0009B689A4201D9FFF7E3BF7047B80D002023
:1010E00010B5084C236820691A68226054600122F8
:1010F00023611A74FFF770FF01462069BDE81040B4
:10110000FFF7FCB8B80D00208260022202740022B2
:1011100042748261704700008368A3F1840243F83F
:10112000142C026943F8442C426943F8402C084AC5
:1011300043F8242CC26843F8182C022203F8102C20
:10114000002203F80F2C43F8082CA3F1200070476D
:101150001503000808B5FFF7DFFFBDE80840FFF7FB
:101160000DBF000010B5202383F31188FFF7D4FFD3
:1011700000210446FFF76CFF002383F3118820460B
:1011800010BD0000024B1B6958610F20FFF734BFF0
:10119000B80D0020202383F31188FFF7F3BF000070
:1011A00008B50146202383F311880820FFF732FF9A
:1011B000002383F3118808BD10B5054C2369036033
:1011C00058610320FFF718FF2369586910BD00BF5D
:1011D000B80D002003682BB1002202605961184647
:1011E000FFF7CCBE7047000049B1064B42681B694F
:1011F00018605A60136043600420FFF70BBF4FF084
:10120000FF307047B80D00200368834206D01A688B
:101210000260506059611846FFF7B0BE7047000089
:1012200038B504460D462068A04206D00368236006
:101230005C604561FFF7A2FEF5E738BD0C3002F0B7
:10124000B5B800000C304FF0FF3302F0AFB800002B
:10125000303002F047B9000030304FF0FF3302F079
:1012600041B900000C3002F07BB800000C304FF0A8
:10127000FF3102F075B80000303002F0F1B8000024
:1012800030304FF0FF3202F0EBB8000001F04ABA04
:1012900037B5154602460B460D4942F8041B044675
:1012A00042600122027204F1540100904FF4806206
:1012B0000C3002F02BF8009404F1300004F2544199
:1012C0004FF480622B4602F0BFF803B030BD00BF80
:1012D000DC38000810B52023044683F3118801F0A0
:1012E00033FA02232372002383F3118810BD000018
:1012F00038B5436904460D461BB90430042101F09A
:1013000099FD04F10C00294602F00EF8002806DAD7
:10131000201D4FF48061BDE8384001F08BBD38BD21
:1013200013B5446BD4F88C341A681178042916D19B
:10133000217A022913D11979128901238B40134292
:101340000DD104F1440001A901F0F6FE024630B1CE
:10135000D4F88C3418681979019B00F0EBF902B0CD
:1013600010BD00000C3001F065BE00000C304FF0E5
:10137000FF3301F05FBE0000443001F04BBF0000BE
:1013800044304FF0FF3301F045BF00000C3001F056
:1013900035BE00000C304FF0FF3101F02FBE0000D1
:1013A000443001F017BF000044304FF0FF3201F02D
:1013B00011BF0000D0F88C2438B5136819780429BF
:1013C000054601D0012038BD017A0229FAD11279EF
:1013D0005C89012090400440F4D105F10C0001F03B
:1013E000C3FD02460028EDD0D5F88C341868597931
:1013F0004FF4807300F08CF9204638BD406BFFF746
:10140000D9BF0000704700007FB50346114A43F87A
:10141000042B04464360012502260F4B0572294622
:101420000193029004F17C0200960C304FF480731B
:1014300001F076FD094B01930096029404F14400FB
:10144000294604F521724FF4807301F051FE04B077
:1014500070BD00BFFC380008FD1300082113000810
:101460000B68202282F311880A7903EB82029061D3
:101470004A79093243F822008A7912B103EB8203D8
:10148000986102230372C0F88C14002383F311883F
:101490007047000038B5044601250430022101F0F0
:1014A000C9FC04F10C0025756FF00101FFF7B8FECF
:1014B00084F84C5004F144006FF00101BDE838405D
:1014C000FFF7AEBE10B501210446043001F0B2FCB6
:1014D0000023237584F84C3010BD000038B5044655
:1014E00000250C3001F034FD04F14400257501F0B5
:1014F00017FE201D84F84C50012101F09BFC204672
:10150000BDE83840FFF756BF90F8443003F0600361
:10151000202B19D190F84520212A0AD0222A4FF0F9
:1015200000030CD0202A0FD1084A82630722C2632D
:1015300007E0064B83630723C363002301E0836353
:10154000C363036401207047002070470108002036
:10155000D0F88C3437B51A681178042904461AD1AA
:10156000017A022917D11979128901238B4013427C
:1015700011D100F14405284601F0AAFE58B101A995
:10158000284601F0D9FDD4F88C3402461979186840
:10159000019B00F0CFF803B030BD000000EB8103E9
:1015A000F7B59C6906460D465CB3202383F311888A
:1015B00006EB8507201D082101F03CFCFB685B69F8
:1015C0001B68443413B1204601F0C4FD204601A934
:1015D00001F0B2FD024618B130462946019B0BE0EE
:1015E000FB685A69116849B11A8A531E0B4005D12C
:1015F0003046294606F1440200F09CF8002383F3AC
:10160000118803B0F0BD0000093110B550F8214039
:10161000CCB1202383F311880421201D01F00AFCA2
:10162000D4F88C241368527903EB820304F10C0084
:10163000DB689B69596801F0A1FC2046FFF7BAFE00
:10164000002383F3118810BD7047000000F0B8BF7D
:10165000034B002258631A610222DA60704700BF10
:10166000000C0040014B0022DA607047000C004083
:10167000014B5863704700BF000C004000F088BB6E
:101680000123037000234360C36183620362C3626A
:1016900043620363038143817047000038B5044609
:1016A000202383F3118800254160C56005614561F1
:1016B000856100F07FFB0223237085F3118838BD1C
:1016C00070B500EB810306465069DA600D4614469A
:1016D00018B100211022FFF7B7FAA06918B1002154
:1016E0001022FFF7B1FA30462946BDE8704000F0FD
:1016F0003BBC0000028902F001020281428902F033
:1017000001024281002202614261826100F0C2BC9A
:10171000F0B500EB81044689E4680125A4698D4099
:101720003543458123600023A2606360BDE8F0403B
:1017300000F0DCBCF0B500EB81040689E46801250B
:1017400064698D403543058123600023A260636096
:10175000BDE8F04000F05ABD70B5022300250446F4
:101760000370A0F84C5080F84E5080F84F5005811F
:101770004581C56005614561856180F8345000F0A0
:101780008FFB63681B6823B120462946BDE8704083
:10179000184770BD436802781B6880F85020052206
:1017A00002700BB10421184770470000436890F89D
:1017B00050201B6802700BB10521184770470000CC
:1017C000F8B50023044680F8343000F1440200F0FC
:1017D00083FC63689B6833B994F8443013F0600667
:1017E00040F0F88005E020469847002840F004814A
:1017F000F2E794F8455003F07F0343EA0525B5F579
:10180000407F3FD010D8022D00F0A88004D845B307
:10181000012D00F09C80DDE0B5F5807F28D0B5F586
:10182000817F00F0B580D5E0B5F5C06F50D008D805
:1018300040F202339D4200F0BC80B5F5A06F2FD07E
:10184000C8E0B5F5106F58D040F602439D427ED0F7
:10185000B5F5006F40F0BE8004F14F03A363012390
:1018600049E004F14C03A3630223E3632564C3E06E
:1018700094F84630012B40F0AD80B4F84C3023F0A2
:10188000020308E094F84630012B40F0A380B4F83E
:101890004C3043F00203A4F84C30A663E66375E0D5
:1018A000B4F84430B3F5A06F0ED194F8463084F804
:1018B0004E30204600F04CFB63681B6813B1204695
:1018C00001219847032323700023A363E36343E0CC
:1018D000626894F8497094F84830556894F8471055
:1018E00094F84620204643EA0723A847002871D0F1
:1018F0004368A3630368E36348E094F84F2094F8D7
:1019000046309A42E0D02378042B10D1202383F371
:1019100011882046FFF7EEFE86F31188636884F88D
:101920004F601B68032121700BB12046984794F843
:101930004630002BC8D084F84F30042323706368EE
:101940001B68002BC0D0204602219847BCE74E4BB5
:10195000A3630223E363002323644DE094F848105B
:1019600011F0800F204601F00F0102D000F0A6FB1D
:1019700001E000F095FB012805D002282AD1434B55
:10198000A363E06302E0424BA363E563266433E0B4
:1019900094F84630F3B994F8483013F00F0193D01F
:1019A0001A06204602D500F0EDFD8DE700F0E0FDBF
:1019B0008AE794F846306BB994F8483013F00F0179
:1019C00082D01B06204602D500F0C8FD7CE700F05F
:1019D000BBFD79E72046002100F0C0FD2046002134
:1019E00000F0B2FD63681B6813B1204606219847DA
:1019F000062384F83430F8BD94F84B2094F84A302C
:101A000043EA0223E26B9A4288BFE36394F94430CD
:101A1000E16B002B0D464FF0200317DA59B101227C
:101A200084F8342083F3118800212046A26BE36BF5
:101A3000FFF780FE16E0032284F8342083F3118838
:101A400020460A460B46FFF763FE19E071B10422F7
:101A500084F8342083F3118800212046A26BE36BC5
:101A6000FFF756FE002383F31188F8BD052284F8A2
:101A7000342083F3118820460A460B46FFF75AFEAE
:101A800085F31188F8BD00BF1C3900082039000813
:101A90002439000838B590F834300446062B46D86F
:101AA000DFE803F0350420353530350090F84B1071
:101AB00090F84A30C26B43EA01239A4212D2C368BB
:101AC0001D8AB2FBF5F305FB13255DB9202383F3D3
:101AD000118829462A462B46FFF72CFE85F31188EC
:101AE000022322E0032384F83430202383F3118877
:101AF00000210B4620460A46FFF70AFE002383F327
:101B0000118838BD036C03B1984700230DE0002114
:101B100000F024FD2046002100F016FD63681B68DC
:101B200013B1204606219847062384F8343038BD87
:101B300090F83420062A38B5044630D80123934063
:101B400013F0670F1BD113F008050FD1DB0626D564
:101B5000052380F83430202383F3118829462A4650
:101B60002B46FFF7E7FD85F3118838BDC3689B69F5
:101B70005B68A3B9036C03B1984700230DE0002113
:101B800000F0ECFC2046002100F0DEFC63681B68DE
:101B900013B1204606219847062384F8343038BD17
:101BA000836D30B5446D9D68002204EB4213013211
:101BB00000214FF0FF30AA42C3F80019C3F81019F2
:101BC000C3F80809C3F8001BC3F8101BC3F8080BBF
:101BD000EBD94FF00113C4F81C3830BD890141F036
:101BE0002001016103699B06FCD4122001F002B9B7
:101BF0002DE9F84F456D0446202383F3118823789F
:101C0000012B04D0236E53B96B69DB0607D4AB6993
:101C100043F01003AB6104F16400FFF7CDFA00213B
:101C200081F31188A36D9B68C8B29842E4D86B69B0
:101C300013F010034ED0676D3B6A03F4F012B2F557
:101C4000802F1DD0B2F5402FF1D1C3F30A1E03F04F
:101C50000F0304EB8303DB681E6A00231A467345F7
:101C6000E5D013F0030F04BF07F580521268072B6D
:101C700098BF327003F101039CBF120A0136EEE7F0
:101C8000C3F30A1803F00F0304EB8303DA689669C1
:101C900096E84410C6EB020E00221646424510D0CC
:101CA00012F0030F04BF07F580563668724538BF3F
:101CB0008CF8006002F101023CBF360A0CF1010C05
:101CC000ECE7DB689B699E6816449E605E68324460
:101CD0005A60ACE70122266E8240324255D020265F
:101CE00086F31188AE6826F00106AE60266E26EAFD
:101CF0000206266683F3118804EB8003D3F80C8078
:101D0000D8F81460D6F80090D6F804E0CE4529D271
:101D1000B8F81070D4F854C0CEEB0903BB4228BF0A
:101D20003B460CEB4017D7F81879BFB2B3EB870FDF
:101D30001AD800F1010B0CEB0B3BD6F808C0E246B9
:101D4000DAF80070CBF80070CAEB03076744042F81
:101D500002D90AF1040AF3E70CEB03077344B760F6
:101D60007360D1E7012000E00020202383F3118875
:101D7000AB6843F00103AB6020B9D5F834381A439F
:101D8000C5F83428002383F3118801314AE70000A5
:101D900010B5064C2046FFF773FC4FF0A04200231D
:101DA0006265034A6366A265A36610BD000E00204B
:101DB0002839000870B50378446D012B86B00546BC
:101DC0005CD12F4B984213D12E4B5A6B42F08002BC
:101DD0005A635A6942F080025A6100225A614320D4
:101DE0000E2101F0CDFB284BE360284BC4F80038EE
:101DF00000232B66C4F8003EC02323604FF4041375
:101E0000A3636E6D202000F0F5FF01233361336979
:101E1000DB07FCD4122000F0EDFF3369002BFCDA65
:101E20000026A6602846FFF7BBFE6B68C4F8106862
:101E3000DB68C4F81468C4F81C680BB9144B00E0E4
:101E4000144BA3614FF0FF336361AB6E93B9124B38
:101E5000009305F17003019305F536730293022395
:101E6000039368460D4B04930595FFF773F9A86635
:101E7000FFF72AF9A36843F00103A36006B070BD21
:101E8000000E0020003802404014004003002002F1
:101E9000003C30C0083C30C034390008F11B000859
:101EA00070B5446D054600212046FFF797FEA96DE9
:101EB00000234FF001128E68C4F83438C4F81C288F
:101EC00004EB43124FF000600133C2F80009B34243
:101ED000C2F8000B4FF0FF30C2F80809C2F8080B37
:101EE000EED90B68EB650B6863626B6D10221A61AB
:101EF0001E6916F01006FBD1122000F07BFFD4F80B
:101F0000003823F4FE63C4F80038A36943F4402387
:101F100043F01003A3610923C4F81038C4F814383F
:101F2000094BEB60094BC4F8106BC4F8003BC4F8D4
:101F30001069C4F80039EB6D03F1100243F480130B
:101F4000EA65A36270BD00BF403900084080001000
:101F5000426D90F84E10D2F8003823F4FE6343EA45
:101F60000113C2F8003870472DE9F0410FB200EBC1
:101F700087080D46D8F80C10446D0E6806F0030370
:101F8000022B07D0032B07D03D4A3E4E012B18BF32
:101F9000164602E03C4E00E03C4E6A01A3184FF0AA
:101FA000000EC3F810EB8B6905F1100C8BB1B1F882
:101FB00012E005F158035B0146EA0E0E44F803E017
:101FC0004FF0010ED4F81C380EFA0CFE4EEA030353
:101FD0000FE004EB471EDEF8003B23F40043CEF88D
:101FE000003BD4F81C384FF0010E0EFA0CFE23EA29
:101FF0000E032244C4F81C380023C2F810394B6980
:1020000005F13F020BB30B8A898B9B08012988BF1E
:102010004B43C16D04EB82025F1841EA0343C7657D
:10202000294653602046FFF7D9FDD8F80C301B8AAB
:1020300043EA85531E4305F148035B01E650012343
:10204000D4F81C28AB40134315E004EB8202104B7C
:10205000536020462946FFF7C1FD04EB4713D3F830
:10206000002922F40042C3F80029D4F81C280123D7
:10207000AB4022EA0303C4F81C38BDE8F08100BF7E
:1020800000800010008004100080081000800C10F8
:1020900000040002826D1268C265FFF781BD000076
:1020A0005831436D49015B5813F4004004D013F4D8
:1020B000001F14BF01200220704700004831436D0B
:1020C00049015B5813F4004004D013F4001F14BFFF
:1020D000012002207047000000EB8101CB68196AE3
:1020E0000B6813604B6853607047000000EB81037E
:1020F00030B5DD68AA691368D36019B9402B84BF75
:102100004023136014686B8A426D013C1C44B4FB8D
:10211000F3F46343E004033340F0C04023F00303CF
:10212000034302EB411009B2C0F8103B2B6803F0E7
:102130000303012B0ED1D2F8083802EB411013F43F
:10214000807FD0F8003B14BF43F0805343F000532E
:10215000C0F8003B02EB4112D2F8003B43F00443CD
:10216000C2F8003B30BD00002DE9F041264D6E6DF8
:1021700006EB40130446D3F8087BC3F8087B380706
:102180000AD5D6F81438190706D505EB8403284676
:10219000DB6821465B689847FA0732D5D6F81438D1
:1021A000DB072ED514B995F8343053B305EB84030F
:1021B000D9688B69C4B94A8A5E68B6FBF2F002FB43
:1021C00010628AB91868DA6890420DD2121A83E850
:1021D0001400202383F311880B482146FFF786FF64
:1021E00084F31188BDE8F0816A890123A34022EAC3
:1021F00003036B81CB6823B121460348BDE8F0415E
:102200001847BDE8F08100BF000E002000EB8103FD
:10221000F0B5DD68436D6A691668D6604C011EB979
:102220001C444FF400220FE019B9402E84BF402017
:10223000106012682F8A42F00056013AD0191C44EF
:10224000B0FBF7F246EAC242C4F810292A6802F04D
:102250000302012A0AB20ED1D3F8080803EB421494
:1022600010F4807FD4F8000914BF40F0805040F093
:102270000050C4F8000903EB4212D2F8000940F004
:102280000440C2F80009D3F8340801228A4002430E
:10229000C3F83428F0BD00002DE9F041274C666DED
:1022A00006EB40130546D3F80879C3F80879F90717
:1022B00026D5D6F81038DA0722D504EB8003D96882
:1022C0004B691868DA6890420FD2121A4FF0000872
:1022D0001A60C3F80480202383F31188204629461E
:1022E000FFF794FF88F311880AE022890123AB40AD
:1022F00022EA030323818B6813B1204629469847BD
:102300003B0618D5D6F834280123AB40134212D02F
:10231000202282F31188226E09481A432266D6F8D9
:10232000342822EA0303C6F834380021FEF752FFAE
:10233000002383F31188BDE8F08100BF000E002068
:10234000640E00207E482DE9F84F446D6369A5694D
:102350001D4015F4805F6561064604D000230366C6
:10236000FFF7FAF9E7E0002D12DAD4F8003E7448DE
:102370009F071EBFD4F8003E23F00303C4F8003EBD
:10238000D4F8043843F00103C4F80438FFF70EFA18
:10239000280504D500236A483366FFF7FBF9A90432
:1023A0000CD5D4F8083813F0060FE36823F4705303
:1023B0000CBF43F4105343F4A053E3602A0704D541
:1023C0007368DB680BB15E489847EB0202D4AF023A
:1023D00057D54DE0D6F854A04FF00009B36D9B6877
:1023E0005FFA89F79F42F2D80AEB4713D3F8002926
:1023F00002F44022B2F5802F37D1D3F80029002A09
:1024000033DAD3F8002942F09042C3F80029D3F818
:102410000029002AFBDB706D3946FFF7DFFB06EB76
:1024200087034FF00108DB6832899B6808FA07F8D8
:102430006FEA080B0BEA0202328113B140483946B9
:102440009847202383F31188DAF834383D480BEAA3
:102450000303CAF83438336E002148EA03033366B5
:10246000FEF7B8FE002383F3118809F10109B5E7EF
:10247000D6F854800027B36D31489B68F9B2994271
:1024800010D9E80629D5202383F31188A3692D48A4
:1024900023F01003A3610021FEF79CFE002383F3C9
:1024A00011881AE008EB4112D2F8003B03F44023F4
:1024B000B3F5802F0FD1D2F8003B002B0BDA428905
:1024C00001238B4022EA0303438100EB8103DB6895
:1024D000DB6803B198470137CDE72903D4F81848E2
:1024E00013D5E20302D50020FFF73EFEA30302D579
:1024F0000120FFF739FE670302D50220FFF734FE03
:10250000260302D50320FFF72FFE6D0313D5E00746
:1025100002D50020FFF7C0FEA10702D50120FFF77A
:10252000BBFE620702D50220FFF7B6FE230702D5E5
:102530000320FFF7B1FEBDE8F84F00F0AFBC00BFCD
:10254000000E0020640E0020436D03EB4111D1F812
:10255000003B43F40013C1F8003B7047436D03EBAD
:102560004111D1F8003943F40013C1F80039704724
:10257000436D03EB4111D1F8003B23F40013C1F884
:10258000003B7047436D03EB4111D1F8003923F450
:102590000013C1F800397047084B1A69920710B54B
:1025A00008D500241C61202383F3118800F0ECFB84
:1025B00084F31188BDE8104000F070BC000C0040AE
:1025C0000D4A136C43F0080313640C4A936843F0FC
:1025D000080393600A4B53229A624FF0FF32DA628B
:1025E00000229A615A63DA605A6001225A613220ED
:1025F0001A60082100F0C4BF00380240002004E047
:10260000000C0040024AD36843F08003D360704757
:1026100000440040F8B5404ED6F85458EF682B6897
:10262000DA059CB20DD5202383F311884FF4007195
:10263000301D00F0FFFB6FF480732B60002383F3E9
:102640001188202383F3118814F02F0321D023074E
:1026500013D014F0080F0CBF00218021E00748BF01
:1026600041F02001A20748BF41F04001630748BF85
:1026700041F48071294800F0DDFBA0066B6896F8F4
:10268000581803D524481940FEF732FE2C68A4B22E
:10269000DAE783F31188390618D5220616D52023E8
:1026A00083F311881E4800F003FF00280ADA1B4854
:1026B000082100F0BFFB4FF63F733B4043F040035F
:1026C000EB6000E06860002383F31188630613D594
:1026D000202383F31188726CB36C0F489A4201D1A6
:1026E000836B9BB94FF6BF733B40EB606FF04003C9
:1026F0002B60002383F31188D6F85C28D3680BB1D4
:1027000010699847BDE8F84000F0C8BB04301021BC
:1027100000F090FBE6E700BFF0100020F41000206E
:102720002011002010B5054C054A20460021FEF777
:10273000AFFD044BC4F8543810BD00BFF0100020AA
:10274000052600080044004038B5234C037A0029D0
:1027500018BF0C46012B0546C0F85C480BD11F4B37
:10276000984208D11E4A136C43F4003313642620A8
:102770000B2100F005FFD5F854381A4A206893421F
:1027800003D002F58062934203D11749B1FBF0F206
:1027900002E0164AB2FBF0F29A60E28842F0400290
:1027A00092B21A61228942F0010292B25A61A28861
:1027B00042F4045141F02C01D96002F4A0520021EE
:1027C0001960B2F5806F19685B680CBF7F23FF2327
:1027D00085F8583838BD00BF64390008F010002073
:1027E000003802400010014000BD010580DE80027B
:1027F00000207047FEE700004FF0FF3070470000F8
:1028000000F002BF08B500F077FB00F07DFABDE8EC
:10281000084000F0F5B8000070470000022906D01B
:10282000032906D00129064818BF00207047054833
:102830007047032A9ABF044B03EBC2000020704785
:10284000783B0008983A00080808002070B5044654
:1028500008460D46FEF7F0F9064620460134037897
:102860003BB12946F2B2FEF7CFF90028F5D101209D
:1028700070BD184670BD00002DE9F04380469BB046
:1028800008460C461646FEF7D7F93849C5B2204629
:10289000FFF7DCFF20463649FFF7D8FF08B11035B7
:1028A000EDB2632D01AF01DC3D4616E0384621460E
:1028B00000F080FF3CE0B9F1250F32D120462B49D2
:1028C0000722FEF7A1F970B92A4B1A682A609A8884
:1028D0009B79AA80AB710734073594F80090B9F161
:1028E000000FE8D122E0204621490822FEF78CF9AA
:1028F000B8B92149AB1C11F8012F20484FEA121E2C
:1029000002F00F021EF800E0125C03F8012C1C4AD2
:1029100003F802EC914203F10203ECD118350834BC
:10292000DBE785F8009001340135D6E785F80090A3
:102930003846FEF781F9C0B2431C5B0088E84800C6
:1029400033700323737002360023DAB2824206F139
:10295000020607D2FA5C06F8022C002206F8012CC7
:102960000133F2E71BB0BDE8F08300BFC43A0008B2
:10297000CC3A0008D53A00080F7AFF1FDD3A00086C
:102980001B7AFF1F08B5202383F311880348FEF745
:10299000DFFD002383F3118808BD00BF601900200C
:1029A00010B50446052924D8DFE801F013230313EA
:1029B000131A202383F3118801210E4AFEF780FEAB
:1029C000204602210C4AFEF77BFE0C48FEF786FDEE
:1029D0000CE0202383F311880848FEF75BFD05E037
:1029E000202383F311880548FEF76CFD002383F351
:1029F000118810BD743A0008A03A00086019002040
:102A000038B50C4D0C4C0D4905F108002246FFF776
:102A100033FF05F1100004F1CA020949FFF72CFF4A
:102A200005F1180004F5CA720649BDE83840FFF701
:102A300023BF00BF08080020101E0020EE3A000847
:102A4000F83A0008CC3A0008BFF34F8F024BDB681E
:102A5000DB03FBD4704700BF003C024008B5094BC4
:102A60001B7873B9FFF7F0FF074B1A69002ABFBF45
:102A7000064A5A6002F188325A601A6822F480626B
:102A80001A6008BDA1200020003C024023016745D8
:102A900008B50B4B1B7893B9FFF7D6FF094B1A69A2
:102AA00042F000421A611A6842F480521A601A68B1
:102AB00022F480521A601A6842F480621A6008BDDB
:102AC000A1200020003C02400B2830B513D80B4A4F
:102AD0000B4C137863B94FF000610A4D44F8231092
:102AE00055F8235001330C2B2944F6D101231370E0
:102AF00054F8200030BD002030BD00BFA0200020D1
:102B000070200020803B0008014B53F820007047E4
:102B1000803B00080C2070470B2810B5044601D9F3
:102B2000002010BDFFF7D0FF064B53F824100A46D3
:102B300043189B1A22B11B680133F1D1043AF7E71D
:102B4000012010BD803B00080B2838B5044621D871
:102B5000114DFFF779FFFFF781FFF323EB60FFF7DC
:102B600073FF0C22B4FBF2F302FB1343DB00DBB276
:102B700043F4007343F002032B612B6943F4803369
:102B80002B61FFF761FFFFF783FF2046BDE8384068
:102B9000FFF7C2BF002038BD003C02402DE9F84FCE
:102BA0001446E207074689466ED42318B3F1016F35
:102BB0006AD2374B1B68DB0766D5FFF74FFF354BF3
:102BC000F322DA60FFF740FF4E46A246C9EB070842
:102BD000BAF1030FB346B04401D8B14624E018F06F
:102BE000030FFAD12B4D2B6923F440732B612B6912
:102BF00043F4007343F001032B613368C8F80030DD
:102C0000BFF34F8FFFF720FFEB6813B1F323EB60A7
:102C10002BE0D8F80080DBF80030984506F1040678
:102C200023D1AAF1040AD1E7C9EB0A033344194DB1
:102C3000C6EB0807012B4F442B691DD923F44073C1
:102C40002B612B6943F4807343F001032B61CB4666
:102C500039F8023B3B80BFF34F8FFFF7F5FE3F880B
:102C6000BBF80030BFB2BB42DED02B6923F00103BA
:102C70002B61FFF70DFF07E023F001032B61FFF746
:102C800007FF2046BDE8F88F4FF0FF30BDE8F88F12
:102C900000380240003C024010B5084C237828B1AF
:102CA00053B9FFF7DBFE0123237010BD23B1207061
:102CB000BDE81040FFF7ECBE10BD00BFA120002012
:102CC000014B186D704700BF002800400A4B1A6F77
:102CD00012045FBF1A6F42F400721A671A6F5CBF6A
:102CE00042F400421A67054A136843F48073136084
:102CF000034B1865704700BF003802400070004069
:102D000000280040FEE7000010B5184CFEF72EF931
:102D1000FEF7A8F800F0A2F8204615498022FEF739
:102D2000F3F9012344F8180C0374124B124AD968C2
:102D300021F4E0610904090C0A431049DA60CA6809
:102D400042F08072CA600E490A6842F001020A60CD
:102D50001022DA77202283F82220002383F31188BF
:102D600062B60848BDE81040FEF7FCB9E00D00204F
:102D7000B03B000800ED00E00003FA05F0ED00E0D4
:102D8000001000E0BC3B0008F8B5184D184B6C690A
:102D9000586A296AA368154A461AB34202F1140612
:102DA00015D80B4421681362B1424FF000034E6006
:102DB000E76851611E46E36001D1FEF753FC86F3DC
:102DC00011882069B847202383F31188DEE7526910
:102DD000B24209D00B441B1A012B98BF022318449E
:102DE000BDE8F840FEF744BCF8BD00BFB80D0020B8
:102DF000000C0040034B59685A68521A8242FBD3B8
:102E0000704700BF001000E083691943037C8161B3
:102E10000A2B03D14369194206D170470B2B07D106
:102E200043691940994203D100234361FEF7A6B8D4
:102E30007047000070B5046805460E46AC420CD0E1
:102E4000E3683343E36016B12269134203D060683C
:102E5000A168FFF7D9FF2468F0E770BD034B044A6F
:102E60001A60044B044A1A60704700BFA422002075
:102E7000A8220020A022002000000220064A536859
:102E800023F001035360EFF30983683383F3098868
:102E9000002383F31188704730EF00E010B5202342
:102EA00083F31188104B5B6813F4006318D0F1EEC4
:102EB000103AEFF309844FF0807344F84C3C0B4B0D
:102EC000DB6844F8083CA4F1680383F30988FEF743
:102ED000DBF808B1064B00E0064B44F8503C10BD4F
:102EE00083F3118810BD00BF00ED00E030EF00E07B
:102EF000250300082803000808B500F057FB074821
:102F000000F00AFCFEF7C2F9FEF7B8FBFEF77AFA0A
:102F1000FFF782FCBDE80840FEF798BB783900084F
:102F200030B5039C0172043304FB0325C361049B89
:102F300003630021059B00604060C1604261026143
:102F40008561046242628162C162436330BD0000F8
:102F50000022416A41610161C2608262C2626FF017
:102F60000101FEF75DB9000003694269934203D194
:102F7000C2680AB100207047181D704710B5046977
:102F80002160C268C3690132C260826923449342EE
:102F9000036124BF436A03610021BDE81040FEF7CE
:102FA00033B9000038B504460D46E36843B9237AC7
:102FB00073B920462946FEF717F90028F5DA09E02B
:102FC00063691A1D1B68A2621344E362002038BDC6
:102FD0006FF0010038BD0000C3684269013BC36067
:102FE000C369134482694361934224BF436A4361C6
:102FF00000238362036B03B11847704738B5054659
:10300000202383F31188846A2CB9FFF7CBFF10B11A
:1030100084F3118838BDAB6AEA6A13F8014BAB62DE
:10302000934202D32846FFF7D7FF002383F311888A
:10303000204638BD2DE9F0471F4604460E4691460E
:10304000202383F31188294B5B6A4FF0000A07EBBA
:103050000308A36A9BB97A1E033202D92046394677
:1030600006E0224A516AC1EB0801B94204D8204661
:10307000FFF798FF18B1002383F3118832E0A16AAB
:10308000E56ACAEB09036D1A9D4228BF1D46402D13
:103090000FD9334601F1400251F8040B43F8040BF9
:1030A0009142F9D1A36A40334036A3620AF1400A43
:1030B00008E030462A46FDF79DFDA36A2B442E44C6
:1030C000A362AA44A26AE36A9A4202D32046FFF7A7
:1030D00083FF002383F31188CA4503D2202383F39F
:1030E0001188B6E75046BDE8F08700BF000C0040ED
:1030F00010B5029C0172043303FB0421C361002359
:103100008362C362039B0363049B00604060C460EE
:1031100042610261816104624262436310BD00004A
:10312000026AC260426A4261026100228262C26235
:103130006FF00101FEF774B8436902699A4203D146
:10314000C2680AB100207047184650F8043B0B6073
:1031500070470000C36842690133C360C369134408
:1031600082694361934224BF436A43610021FEF7B1
:103170004BB8000038B504460D46E36843B9237ADE
:1031800073B920462946FEF72FF80028F5DA09E042
:103190002269131DA362E3691344E362002038BD72
:1031A0006FF0010038BD000010B504692160C268ED
:1031B000C369013AC260826923449342036124BF18
:1031C000436A036100238362036B13B1BDE81040BF
:1031D000184710BD70B5202304460E4683F31188AE
:1031E000856A35B91146FFF7C5FF10B185F311881F
:1031F00070BDA36A1E70A36AE26A01339342A362A0
:1032000004D3E16920460439FFF7CEFF002080F3A4
:10321000118870BD2DE9F0471F4604460D469146C2
:10322000202383F31188294B5B6A4FF0000A07EBD8
:103230000308A36A9BB97A1E033202D92046394695
:1032400006E0224A516AC1EB0801B94204D820467F
:10325000FFF790FF18B1002383F3118832E0A06AD2
:10326000E66ACAEB0903361A9E4228BF1E46402E64
:103270000DD905F1400355F8042B40F8042B9D426D
:10328000F9D1A36A4033A3620AF1400A08E0294653
:103290003246FDF7AFFCA36A33443544A362B2441F
:1032A000A26AE36A9A4204D3E16920460439FFF72F
:1032B0007BFF002383F31188CA4503D2202383F3C5
:1032C0001188B6E75046BDE8F08700BF000C00400B
:1032D000026943699A4203D1C3680BB1836A0BB98F
:1032E00000207047043B9B1AFAD01360C368013B6F
:1032F000C360C3691A44836902619A4224BF436A66
:1033000003610023836201207047000010B50A4466
:103310000024C361029B006040608460C1608161E1
:1033200041610261036210BD08B58269436993423D
:1033300004D1826812B14FF0FF3008BD82680132BB
:1033400082605A1C42611970426903699A4201D332
:10335000C36843610021FDF757FF002008BD00004E
:1033600070B5202304460E4683F31188A56845B93D
:1033700020463146FDF738FF0028F7DA85F311883B
:1033800070BDA368A269013BA360531CA3611578BB
:103390002269934224BFE368A361E3690BB120462D
:1033A0009847002383F31188284670BD2DE9F84F14
:1033B0001D4604468A469046D0F81C90202383F38D
:1033C0001188204B5F6A00262F44A3689BB96A1EB0
:1033D000033202D92046294605E01A4A516A791A71
:1033E000A94205D82046FDF7FFFE0028EDD00023B6
:1033F00083F3118822E0A368013BA360A3695A1CF0
:10340000A2611B788AF800302369A2699A4224BF1E
:10341000E368A3610AF1010BB9F1000F01D0204666
:10342000C847002383F31188B8F1010806F10106AB
:1034300004D0202383F31188DA46C6E73046BDE87E
:10344000F88F00BF000C00408260C3610A44009BFB
:1034500000604060C1608161416102610362704748
:10346000F8B504460E461746202383F31188A56855
:1034700045B920463946FDF7B7FE0028F7DA85F34F
:103480001188F8BDA368013BA36063695A1C62619F
:103490001E70236962699A4224BFE3686361E3692D
:1034A0000BB120469847002080F31188F8BD00003A
:1034B000836942699A4210B504D1826812B14FF013
:1034C000FF3010BD8268013282605A1C82611C7814
:1034D00003699A4201D3C36883610021FDF794FE1A
:1034E000204610BD2DE9F84F1D4604468A469046F9
:1034F000D0F81C90202383F31188204B5F6A0026AC
:103500002F44A3689BB96A1E033202D9204629467C
:1035100005E01A4A516A791AA94205D82046FDF7F2
:1035200063FE0028EDD0002383F3118822E0A36816
:10353000013BA36063695A1C62619AF800201A700B
:10354000236962699A4224BFE36863610AF1010B4F
:10355000B9F1000F01D02046C847002383F311883A
:10356000B8F1010806F1010604D0202383F3118885
:10357000DA46C6E73046BDE8F88F00BF000C0040D1
:1035800000F1604300F01F02400903F561430901A7
:103590008000C9B200F1604083F8001300F561407B
:1035A00001239340C0F8803103607047144B002121
:1035B0001A694FF0FF321A61196158695A615961ED
:1035C000186A60F0805018621962586A5A6259622B
:1035D0001A6C42F080521A640A4A106840F48070F3
:1035E0001060186F00F44070B0F5007F1EBF4FF4FC
:1035F000803018671967536823F40073536070476D
:103600000038024000700040324B4FF080521A6484
:10361000314A4FF4404111601A6842F001021A60C9
:1036200019682C4A8807FBD5936823F0030393603D
:1036300093689360274B9A6812F00C02FAD11968CC
:1036400001F0F90119609A601A6842F480321A6038
:103650001968204A8903FBD5536F43F00103536770
:103660001C4B5A6F9007FBD51C4A5A601A6842F0EF
:1036700080721A60184B5B685904FBD5154B1A68A9
:103680009201FBD5164A9A60164B1A68164B9A425D
:10369000164B07D1164A1168164A914202D140F2E0
:1036A000051201E040F205721A600A4B9A6842F076
:1036B00002029A609968074A01F00C010829F9D1C1
:1036C000536C43F480435364536E43F48043536616
:1036D000704700BF003802400070004008544007A7
:1036E00000948838002004E011640020003C02406F
:1036F00000ED00E041C20F414B6843608B6883607E
:10370000CB68C3600B6943614B6903628B69436299
:103710000B680360704700001C4B196B40F2FF12EE
:10372000114310B51963196D04460A431A65214601
:103730001748FFF7E1FF04F11C011648FFF7DCFF13
:1037400004F138011448FFF7D7FF04F1540113487E
:10375000FFF7D2FF04F170011148FFF7CDFF04F12C
:103760008C011048FFF7C8FF04F1A8010E48FFF7CD
:10377000C3FF04F1C4010D48FFF7BEFF04F1E001EF
:103780000B48BDE81040FFF7B7BF00BF003802404C
:10379000000002400004024000080240000C024009
:1037A000001002400014024000180240001C0240B9
:1037B0000020024080EA0102844612F0030F4FD13C
:1037C00011F0030F32D14DF8044D11F0040F51F8F0
:1037D000043B0BD0A3F101329A4312F0803F04BFA7
:1037E0004CF8043B51F8043B16D100BF51F8044B90
:1037F000A3F101329A4312F0803FA4F101320BD1C0
:103800004CF8043BA24312F0803F04BF51F8043B44
:103810004CF8044BEAD023460CF8013B13F0FF0FA1
:103820004FEA3323F8D15DF8044B704711F0010FD4
:1038300006D011F8012B0CF8012B002A08BF7047A5
:1038400011F0020FBFD031F8022B12F0FF0F16BF9C
:103850002CF8022B8CF8002012F47F4FB3D1704764
:1038600011F8012B0CF8012B002AF9D1704700BF89
:10387000121012131211000060190020F010002025
:1038800000000000B03800083F00000013040000F2
:10389000BA3800083F00000019040000C4380008CE
:1038A0003F00000021040000CE3800083F00000067
:1038B00053544D3332463F3F3F0053544D3332460D
:1038C0003430780053544D333246343278005354F8
:1038D0004D3332463434365858000000591200082F
:1038E00045120008811200086D12000879120008C4
:1038F00065120008511200083D12000881130008EB
:103900006D130008A913000895130008A1130008FF
:103910008D130008791300086513000800000000EB
:1039200000000000010000008000000040010000D5
:10393000030000007573625F70756D700000000019
:1039400000000000C1170008951A0008311B00088C
:1039500040004000D8100020D810002001000000D6
:10396000E8100020009600000000000000000000A9
:1039700000000000000000000000802A000000009D
:10398000AAAAAAAA00000000FFFF00000000000091
:1039900000A00A000000000000000000AAAAAAAAD5
:1039A00000000000FFFF0000000000000000000019
:1039B0000000000000000000AAAAAAAA000000005F
:1039C000FFFF0000000000000000000000280000D1
:1039D00000000000AAAAAAAA00140000FFFF00002D
:1039E0000000700700000000500000000000000010
:1039F000AAAAAAAA00000000FFFF00000000000021
:103A0000000000000000000000000000AAAAAAAA0E
:103A100000000000FFFF00000000000000000000A8
:103A20000000000000000000AAAAAAAA00000000EE
:103A3000FFFF000000000000000000000000000088
:103A4000000000000A000000000000000300000069
:103A50000000000000000000000000000000000066
:103A60000000000000000000000000000000000056
:103A70000000000002000000000000009D1500088A
:103A80000916000840004000F01D0020001E002024
:103A9000020000000000000043000000143B00088A
:103AA00003000000000000004916000800000000AC
:103AB000100000005019002000000000010000006C
:103AC0000000000025424F41524425002553455235
:103AD00049414C2500663462792D636800303132EB
:103AE0003334353637383941424344454600417214
:103AF000647550696C6F740025424F415244252D06
:103B0000424C0000A12900081D28000809150008E2
:103B10008529000809024300020100C0320904009F
:103B2000000102020100052400100105240100012A
:103B3000042402020524060001070582030800FF91
:103B400009040100020A000000070501024000000C
:103B50000705810240000000120110010200004030
:103B6000830440570002010203010000040309041A
:103B7000000E00200101020012000000583B000866
:103B80000040000000400000004000000040000035
:103B9000000001000000020000000200000002001E
:103BA000000002000000020000000200000002000D
:103BB0006D61696E0069646C65000000B53B0008CA
:103BC000A8200020A022002001000000052D0008F0
:103BD0000000000000000000FF0096000000000848
:103BE000040000006C3B0008000000000000000022
:103BF00000000000000000000000000000000000C5
:00000001FF
